:1000000083018B018A01850186018C019D018F018D
:100010009001910192019301940195019801990138
:100020009A01831610308500003086008117640025
:10003000A73081008312850127309E009F019F0B0E
:100040001F289E0B1F2838304B2008304B200130D2
:100050004B200C304B2006304B20BD288316FF3040
:1000600086001830850083120510851405150608D2
:1000700005118039031D2E28851083160030860057
:100080008312080096002E20851005140515160809
:1000900086000511080096002E2085100510051514
:1000A00016088600051108009B010C089C00AA2078
:1000B00003149802031867280314013099020318E7
:1000C0006728031401309A02031867281B149C0345
:1000D0001C08AA2003149902031874280314013081
:1000E0009A02031874281B149C031C08AA200314EA
:1000F0009A0203187D2803147E281B0C00349B01F0
:100100000C089C00AA2003109807031C92280310D7
:1001100001309907031C9228031001309A07031C31
:1001200092281B149C031C08AA2003109907031C87
:100130009F28031001309A07031C9F281B149C035F
:100140001C08AA2003149A07031CA8280314A92832
:100150001B0C00348207003400340A3400340034AD
:10016000643400340334E834003427341034013468
:100170008634A0340F344234403411308C000930BE
:100180008D008E0106309D0054200318CE288E0A63
:100190008D03031DC42803308C02D1287F20033037
:1001A0008C0209308D0010301D079B009B031B083B
:1001B00084000E088E0180009D0301300C07031D92
:1001C000C42818088F0006309D00003080384B206E
:1001D0000F301D0784000008303842200530031519
:1001E0001D02031DF5282E3042209D0BE8280F30FC
:1001F0001D078400000830384220403080384B20F2
:10020000203042204D304220483042207A30422077
:10021000003080384B2097018101000000009D01D3
:100220000B309E0001309F00D530A0008B011030B4
:10023000850083161F30850083120B1D2229970A23
:100240000B1125290000000000009E0B1D290B301A
:100250009E009F0B1D2901309F00A00B1D29F4302B
:100260008E000B1D3629970A0B113929000000005A
:1002700000008E0B3129000000000000000000008B
:10028000000000000000000003018600103085001F
:1002900083161730850083120108990017089A0009
:1002A0009B019B0A851585110B1101080311190289
:1002B000031951299B0A9B099B0A1B0A9800BD2818
:00000001FF
